:02000000D32803
:1000080009008A0123088207D229D329D329D329B1
:10001800D329D329D329D329D329D6298A01230837
:100028008207FC29F829DF29E829F829F829F8297D
:10003800F629D929FC298A01230882071E2A182AA9
:10004800162A182A162A162A0F2A082A182A072AC8
:100058008A0182070D34EA282034EE281A346229EE
:100068004134122955342A2B5334E12B5234F02BC6
:100078004434ED2A5034012C4C34652951343E2C3B
:100088002F34C92B4634D52B2D34CF2B2E34402971
:100098002C3447293D344E293B345E295B34DB2D13
:1000A8005D34EC2D3F341B2900348A0182000D3465
:1000B8000A345634653472347334203433342E346D
:1000C8003334203441346C3467343D3400340D34D7
:1000D8000A345534503450343E3400340D340A3424
:1000E800503472346F346734003443346F346E34B0
:1000F8006634693467340A3400340D340A345334AE
:1001080074346F34703400340D340A345234753416
:100118006E34003443346834653463346B340034EB
:100128000D340A344C346F34613464340034203470
:10013800503472346F3467342134003420345334EB
:100148006B346934703421340034203443346F34D0
:100158006E34663469346734213400340D340A341B
:1001680044346134743461343D34003420344534CB
:10017800723472346F347234003420342D342034A5
:10018800413462346F3472347434003420344F3460
:100198004B34003443346F3472346534003483167E
:1001A80000308500023086008030810014309200D3
:1001B800831236250C3097000430920007309F00D8
:1001C8000A30CA001B2134210520E3236B30C023E9
:1001D800A014F8242425DC00E60166082C20003A47
:1001E800031909295C060319FC28E60AE60AF1281E
:1001F800E60A66082C20EE288E3003299430C023A6
:10020800BA30C023C130C0230C29DC233F304B2532
:10021800E323EA28DC23AC24DB24080001305A2538
:100228007724D900093C031C092959085E255B304D
:10023800C02301306A25A300902403306A25A20058
:10024800463022184B252F304B2502306A25C9002D
:1002580090242D304B2504306A25CA0090240800CC
:100268002308093C0318080000301221A2011430A9
:10027800C9230030D5230800AC245908201FA7251E
:10028800201BFA250800AC245A08E2005908E100AE
:1002980094250800B230C023201F56291B262E267D
:1002A800E02408000430A7259D256208E0246108A1
:1002B800E0240800AC24590830240800FF3012213B
:1002C8000800E323323030249430C023201B7B2ADB
:1002D80005240A303024AD01AE011220E323323068
:1002E800302405241430302454247C29A2307D295C
:1002F8009B30C0239A224D08CC000310CC0CCD01B2
:100308002C083F3C031C8D299322BD211F206A2401
:100318007C29DC2393222C08403A031D7A292B08D8
:100328000E3A031D7A295922A930C0239A22DC23C8
:100338009322A230C0234D08031D9A29DC238E3056
:10034800C023E3236430302405242908D9002A086F
:10035800DA0056247025D903590FDA0ADA03590846
:100368005A04031DAE297024BA300319CA30C023B9
:100378000C292E082C06031DC6292D082B06031D43
:10038800C6290800FF30E1003F30E2005A24063059
:10039800A725AD0AAD0A0319AE0ABD290800201326
:1003A800A01308002017A0170800FF210930A7256F
:1003B8000830A725FA29FD2157225722572257220C
:1003C800572257225722E929FF210130A725073054
:1003D800A7250830A7250A3030240130A725073083
:1003E800A725FA291F30F9290930A7251430302408
:1003F80008000030002A0230A7253F30E200FF3015
:10040800E100942508007B2A0130D4001830D2007E
:100418001730D300332A0230D4001830D2000A3003
:10042800D3001F2A0430192A0A30D4000830D20019
:10043800D3011F2A08000230A725C922E1008E2215
:10044800C922E2008E2294255208A7255408302498
:100458005308031DA7255722CC0B1F2A080020127A
:10046800462257224622572246225722462252081F
:10047800A725540830245308031DA7255722201EFA
:10048800342A08000230A725C922201AFF30E100CB
:100498008E22C922201A3F30E2008E229425CC0BEE
:1004A8000800201608000630A72D0030A725E20115
:1004B800E1019425AD012D082B060319682A0630A1
:1004C800A725AD0AAD0A5F2AC922E100C922E200C8
:1004D8000230A72594255208A7255408302453082C
:1004E800031DA7250630A725CC0B682A0800F4238E
:1004F80021304B259A224D08CC0003190800CD0164
:10050800CF25C922FA25CC0B852AEC2507303024C3
:1005180093227C2AAD0A031D0800AE0A08000D309C
:100528004B252C08E0242B08E0240800EA24242585
:100538003A3A0319A42A3A3A0D3A031D9B2A02298A
:10054800CD01DB01BE22CF00BE22AC00BE22AB0033
:10055800BE22CF080319B42ABE22C122CF0BB02A6B
:10056800BF24003CDB06031908003D304B255B081F
:10057800E0240029BF24DB070800DC0031304D07E8
:1005880084005C088000CD0A080031304D078400E3
:100598000008CD0A0800201FD52AF423CF25D72527
:1005A800080005240800201FE22A1030CC00CD01E5
:1005B8001B262E26C122CC0BDC2A08000830CC00D2
:1005C800CD0170256208C1226108C122CC0BE52A41
:1005D8000800AB01AC01CF222010D7220830CC0094
:1005E800CD01DC232C08E0242B08E0243A304B25ED
:1005F80020304B25C922E024C922E024CC0BFC2A58
:1006080020304B250830CC00CD01C922A01F0E2B6D
:1006180024234B25C92224234B25CC0B092B3F250A
:10062800201C1D2B422542252010DC001B3A0319F3
:1006380006291030A01F0830AB070318AC0AF12AAE
:100648007F39E03E203E03182E300800201B632B24
:10065800AC24B6237C2305243230302420102F0804
:1006680030040319482B86230830DF007025610801
:10067800DB07E0246208DB07E024DF0B3A2B5B088A
:10068800003CE0249723332BDC233A304B25DB0155
:100698000230DB07E0244030DB07E0240E30DB07C4
:1006A800E0240030E02483256108DB07E0246208A9
:1006B800DB07E0245B08003CE024A4230C29AC24DD
:1006C800B3237C23CF2220102F08300403197A2B60
:1006D80086231030DF001B262E26DB07E024DF0BE5
:1006E8006F2B5B08003CE0249723682BA4230C297C
:1006F8005908013E0318DA0AAF005A08B000AB01E6
:10070800AC010800DC233A304B25DB011030DB0755
:10071800E0242C08DB07E0242B08DB07E02400306A
:10072800DB07E02408002B08103E0318AC0AAB00D6
:100738003F2520180629AF080319B003AF030800A6
:10074800DC233A304B250030E0240030E024003030
:10075800E0240130E024FF30E024DC23080003100B
:10076800DA0CD90C0310DA0CD90C0310DA0CD90CFA
:100778000310DA0CD90C0800E30063085920003A8A
:10078800031908004B25E30AC12B02305A257724A8
:10079800C9005E251B2904305A257724CA005E2526
:1007A8001B290130A20603305A2522085E251B2981
:1007B8000D304B250A304B2508008130C0232324F7
:1007C800061605100A3030242C240A3030248316EB
:1007D80085140515831208008830C023F423080007
:1007E80023241430302427240A3030248316851417
:1007F800051583120612051408007230C02305245B
:100808000800061683168510051183128510051138
:10081800053030241F241430302427243230221C81
:100828003024061205140A303024080042251B3AE9
:10083800031D1A2C08000A309500851508000030A1
:100848009500851108008617831686138312080001
:100858008316861783120800EB005C30EA000A3022
:10086800E900861C2014E90B352CEA0B332CEB0B22
:10087800312C0800CE30C02384011030EC00103039
:10088800ED00DC230408E0243A304B2520304B25CA
:100898000008E024840AED0B4A2CEC0B432C0800DA
:1008A800A901AA01A501A601A0160800A01E08001A
:1008B80061083F39A5066208A6060310A50DA60D16
:1008C80003182514A90A0319AA0A08002508A7006D
:1008D8002608A800A012080025082706031D0800FE
:1008E800260828060800DD012425DC003030DC025B
:1008F800031C862C0A305C020318862C89245C08A9
:10090800DD07782C2A255D0808000310DD0D5D0839
:10091800DD0DDD0DDD070800A110DD006430982431
:100928000A309824A1140130DC003030A4005C089F
:10093800DD02031CA12CA40A9C2CDD072408A118A5
:100948004B2D303A031DA114303AA1184B2508004D
:100958000430E600DA01D901C5240318BD2CD90DED
:10096800DA0DD90DDA0DD90DDA0DD90DDA0DD90751
:10097800B02C2A250800C524DC00DC0EC5245C0741
:1009880008002425C8240800D03E031CD42CF63EB9
:10099800031CD82CF93E031CD42CFA3E031CD72C7C
:1009A800031400300800063E0A3E031008005A08E7
:1009B800E0245908E0240800DD005D0EE4245D0809
:1009C8000F39F63E0318073E3A3E4B2DA0308400FF
:1009D800D10142258000840A0D3A031908000D3A16
:1009E8001B3A03190629ED2CD10142252C25DE00DE
:1009F8000A3A0319F92C5E08083A0319142D51080C
:100A0800A03E84005E088000A0184B255E080D3AC1
:100A18000319222DD10A51084D3A03191E2DF92C1C
:100A2800D103D11BF82C08304B2520304B2508303A
:100A38004B25F92C08304B25D103F92CD10108009E
:100A48005108A03E84000008D10A0800D10308001C
:100A58009F3E031C342DE63E0318203E5B3E0800F3
:100A6800613E0800831624309800403099008312B4
:100A78009030980008008C1A20140800981C462D05
:100A8800181218168C1E462D8C121A0808000C1EF7
:100A98004B2DDC004A08031D30245C0899000A3AF3
:100AA800031D08004908013E3024080083169B00F6
:100AB8008312080083161C159A0055309D00AA3031
:100AC8009D009C149C18662D8312080083169B00B9
:100AD8001C141A08831208000430A7259D25063027
:100AE800A725080088250230A7255A08E2005908DA
:100AF800E10094250830A7250A303024080088250D
:100B08000430A7259D2508000030A725E101E20152
:100B180094250730CC000630A725CC0B8F2D080074
:100B28005A240310E10DE20D6108AA256208AA25DE
:100B38000800BC25E100BC25E2000310E20CE10C32
:100B480062135A240800DC000630AC2DDC000830A3
:100B5800D60083168510831205155C1885145C1C55
:100B68008510DC0C000000000511D60BB02D080024
:100B78000830D600831685148312DC010515DC0CB9
:100B8800DC1305110000000000008518DC17D60BE7
:100B9800C22D5C080800DB25A030FA252C08FA25B0
:100BA8002B08FA250800DB25A130FA250800831652
:100BB80005118312051100008316851483120000A5
:100BC800051585108316851083120000051108008D
:100BD8000511851083168510831200000515000085
:100BE800831685148312000005110800DC00083004
:100BF800E600DC0D8510831603188514031C851088
:100C0800831200000515000000000511E60BFD2DFC
:100C18008316851483120000000005150000851C4A
:100C2800182E05112114080021100511080008309C
:100C3800E600831685148312051500000310851835
:100C480003140511DC0D000000000000E60B202E47
:100C58005C080800851083168510831205150000AE
:100C6800000000000511080083168514831205157D
:0A0C78000000000000000511080054
:02400E00223F4F
:00000001FF
